:1070000061C00000A0C0000084C0000082C0000079
:1070100080C000007EC000007CC000007AC000007C
:1070200078C0000076C0000074C0000072C000008C
:1070300070C000006EC000006CC000006AC000009C
:1070400068C0000066C0000064C0000062C00000AC
:1070500060C00000EC2DFD2DB7B6B0FCFDCF27BF02
:10706000E895B7B6B0FCFDCF21E1B7B6B6FCF4CFDA
:107070000895090212000101008032090400000095
:107080000000000012011001FF000008C016DC051E
:107090000201010200010E0355005300420061008D
:1070A000730070001C037700770077002E006600E5
:1070B00069007300630068006C002E0064006500C6
:1070C0000403090411241FBECFE5D8E0DEBFCDBF05
:1070D00024B7D8E0CEE539913833399109F03FEF44
:1070E00030939C0020939B0010E0A0E6B0E0E4E623
:1070F000F8E702C005900D92A636B107D9F720E057
:10710000A6E6B0E001C01D92AB39B207E1F778D135
:10711000A7C376CFA82FB92F80E090E041E050EAD6
:10712000609530E009C02D9182279795879510F0E2
:1071300084279527305EC8F36F5FA8F30895EADFD0
:107140008D939D930895CF93CFB7CF93DF93C3953E
:10715000849BE9F7849B0BC0849B09C0849B07C078
:10716000849B05C0849B03C0849B01C089C06F932E
:10717000C0917E00DD27CB57DF4F2F9365E5849BC1
:1071800003C02F916F91E6CF0F931F934F9320E091
:1071900040E15F9300B3047104FB27F93F9350E093
:1071A0003BE039C0147140642F77012F5F5F1EC030
:1071B000406810B314712F7752501FC0406400B361
:1071C0002F770471D1F15F5F00C023C0406210B31C
:1071D0002F77147191F15F5F00C025C004711027F3
:1071E000515012F45D5F0000115027952C3F10B3F1
:1071F000C8F614710127015027952C3FC8F6422785
:10720000499300B3047110274F73115027952C3FF9
:10721000A8F64695469510B3147179F001270150F0
:1072200027952C3F98F66B5A60F3315000B3B0F6B7
:1072300000C010E41ABF002717C03B503195C31B94
:10724000D04010E41ABF0881033CF9F00B34E9F098
:1072500020917C001981110F1213EDCF093651F1E5
:107260000D3211F0013E39F7009383003F915F9199
:107270004F911F910F912F916F91CAB7C6FD67CFA4
:10728000DF91CF91CFBFCF9118952091830022231A
:1072900069F310918100112339F534303AF13093BC
:1072A000810020937D0010917E003BE0311B3093E4
:1072B0007E001CC0009181000130B4F40AE53091D9
:1072C000610034FD14C000936100C1E7D0E013C039
:1072D000052710E000C0000002BB1AC0052710E01F
:1072E000221F1DC010E021C04AE502C032ED432F2D
:1072F000C4E1D0E032E011B31461949A02B311BB3F
:1073000054E120E865E320FF052702BB2795179588
:107310001C3FF0F66695B8F7B1F720FF052702BBD2
:10732000279517951C3FD0F62795179517FF05272A
:1073300000001C3F02BBB0F629913A9519F70B7E6D
:1073400010918200110FC651D04002BB11F0109372
:107350007C0010E41ABF006111B31B7E402F4B7EEE
:1073600054E05A95F1F702BB11BB42BB7FCFDC0161
:1073700013963C911397932F1496EC9114978E2F9C
:1073800012962C911297203331F4E370F0E0EE590D
:10739000FF4F80810895283529F431110EC0E1E0B6
:1073A000F0E006C0203571F4311128C0E0E0F0E0D3
:1073B00089E080935700849108953830F9F4E3E030
:1073C000F0E0F6CF203221F4FC01EE0FFF1F06C0E3
:1073D000283231F4880F991FFC0131968491089569
:1073E000203A09F428C2203C21F415966C912BD246
:1073F00005C02F3F19F481EF80936F0080E008955E
:1074000011BA80E882BB81E08BBF82E08BBFE0E0F5
:10741000F1E7A89531978040E1F780919B00877F45
:1074200021F480919C00882369F0879B0BC0F8941D
:107430008C9A12BA1BBE15BE81E08BBF1BBEE0E06A
:10744000F0E009958EEF80936F0014BE0FB6F894AC
:10745000A89581B5886181BD11BC0FBE85B78260DA
:1074600085BF8BB780648BBF8C9A8CE0E0E0F5E33E
:10747000A89531978040E1F78C987894109181001D
:10748000135017FD41C180917E00CCE0D0E0C81BB5
:10749000D109CB57DF4F80917D008D3209F0B8C004
:1074A000183009F02FC183EC809371008AE5809336
:1074B0006100109270003881832F80769981882333
:1074C000C1F146E650E05093800040937F00933036
:1074D00031F4CE014CDF8093690084E08FC0953099
:1074E00009F48BC09A3009F488C08CEF890F86307C
:1074F000B0F44A815B8150936E0040936D009930E7
:1075000009F491C18E8180936C002D8122702093AB
:107510006B0090936A0037FD6CC08FEF6AC080915A
:107520006F00923011F48E7F01C0816080936F00F4
:107530007AC18A8110927A00911106C010927B0064
:107540002AE730E082E050C0953019F48093820041
:107550003DC09630A9F59B81913019F484E890E7FD
:1075600004C0923041F482E790E7909380008093CA
:107570007F0082E121C09330F1F4811108C080ECDA
:1075800090E79093800080937F0084E015C0813065
:1075900041F484EA90E79093800080937F008CE12F
:1075A0000BC0823041F486E990E79093800080938D
:1075B0007F008EE001C080E090E4909370001EC0D8
:1075C000983079F0993031F4809384002AE730E0E4
:1075D00080E00AC081E09A3009F080E02AE730E0DC
:1075E00003C024E830E081E03093800020937F00E6
:1075F00005C090E89093700008C081E09F819111D0
:1076000004C09E81981708F4892F809360007AC087
:107610008091700087FF76C000916C00011708F41C
:10762000102F011B00936C00F12CF11608F066C0BE
:1076300020916A0080916D0090916E00273080F05B
:107640006E01FFEFCF1ADF0A68819C012F5F3F4F69
:1076500030936E0020936D00F6D0F394E601E5CFF1
:107660008115904708F04CC0F394F394F894E0919E
:107670006D00F0916E002991399181E009018093AC
:107680005700E8951124789480916D0090916E00D8
:10769000029690936E0080936D008F779927892BC7
:1076A00051F00111C2CFF11608F4BFCF80916B00E9
:1076B000882309F4BACFF894E0916D00F0916E0040
:1076C000329783E080935700E895789407B600FCE2
:1076D000FDCFF894E0916D00F0916E00329785E057
:1076E00080935700E895789407B600FCFDCFF89496
:1076F00081E180935700E895789497CF011102C0FB
:1077000010926000109281008091610084FF67C038
:10771000809160008F3F09F462C0C82F893008F063
:10772000C8E08C1B809360009091710088E88927E5
:1077300080937100CC2309F478C08091700087FF9A
:107740002AC080916C008C1708F4C82F8C1B809382
:107750006C00D0906A00D0E082E7E82E80E0F82E3E
:10776000CD1789F100916D0010916E0086E08D15A6
:1077700018F4C80160D002C0F8018491F701808339
:10778000FFEFEF1AFF0A0F5F1F4F10936E00009379
:107790006D00DF5FE5CFE0917F00F0918000A2E710
:1077A000B0E086FF07C08C2F94919D933196815055
:1077B000D9F705C08C2F91919D938150E1F7F093FB
:1077C0008000E0937F006C2F82E790E0B8DCCC5F14
:1077D000CC3019F08FEF80936000C093610084E19A
:1077E00090B3947131F48150D9F7109282001092C5
:1077F0007C0080916F00803130F0879B0FC08091BA
:107800006F00805109C0879909C080916F00823054
:1078100028F080916F00825080936F0080916F00FC
:1078200081112CCE04CE80E0E9CE60E082E790E0CA
:1078300086DCC4E0CFCFE199FECF9FBB8EBBE09A40
:1078400099278DB30895262FE199FECF9FBB8EBB5C
:107850002DBB0FB6F894E29AE19A0FBE01960895F7
:04786000F894FFCFCA
:06786400FF5A1E95020010
:040000030000700089
:00000001FF
